:030000000219FDE5
:03000B000200AA46
:03002B000201636C
:03005B000202F2AC
:030073000202DFA7
:1000800002030406080C10182030406080040608A3
:100090000C10182030406080A0C00003070F1F0D17
:1000A0000D0403060D0503030202C2AFC0D0C0E079
:1000B000206214E5256009E473E525F4F58AD2622F
:1000C000D0E0D0D0D2AF3285268AC262E526F46075
:1000D0003630682C20720DD0E0D0D0C283C294C2DA
:1000E00095D2AF32C283C294C295206F132066109E
:1000F000740CD5E0FDE57BB50704429021004280F9
:10010000D0E0D0D0D2AF32758A00C28DD262210049
:1001100001B9306805206602D28301B93068052034
:100120006602D29401B9306805206602D29501B901
:10013000C28030680A2066077408D5E0FDD28301CA
:10014000B9C28230680A2066077408D5E0FDD294EF
:1001500001B9C29730680A2066077408D5E0FDD25D
:100160009501B9C2AFC2AD53E6EFC0D0C0E0D2D363
:10017000D2AFC2CEE52A6007207449152A21C4787F
:1001800000790020742EE580307E01F430E502789D
:10019000FF53DACF207E0343DA20307E0343DA10A8
:1001A000C2D8C271E580307E01F430E50279FFC328
:1001B000E89970CB306103752A40207403752A409A
:1001C000885CD27020740DE52B6004152B21D4437C
:1001D000DA01C2D820700221E7A85C206102C27057
:1001E00020740221E588227882B60403852224C384
:1001F000E52594404002D26420CF0AD0E0D0D0431D
:10020000E610D2AD32C2CF053A7802E52A60053059
:100210007402152AC3E55C94014005755F00413105
:10022000756000756900E55F2401F55F5003755F37
:10023000FF7982B7020D306E1DC3E522943240165D
:10024000854C227982B7030E306E0BC3E5229432BF
:100250004004798E8722C3E5239522600840041567
:100260002341650523D8CA0569E56970021569D57A
:100270006A63756A017805C3E569956B4057C3E504
:1002800069956C50087801756A03020299C3E569A3
:10029000956D50057801756A01C3E5629524401E8D
:1002A0007982B7040241CA206E14852462E569048C
:1002B0006003856B69756A0175233C0202D5E562AE
:1002C0002850057562FF41CAF562E5620470067543
:1002D00060FF7569FFD0E0D0D043E610D2AD32C2E6
:1002E000AF53E67F7592FA7593FFC260759104D2A1
:1002F000AF32C2AF53E6EFC2ADC0D0C0E0C0F0D263
:10030000D3D2AFA8FBA9FCC2D8307102615953DA2D
:10031000CF207E0343DA10307E0343DA20D271E52A
:1003200080307E01F420E502613088278928A13ED3
:1003300053DACF207E0343DA20307E0343DA10C243
:10034000D8C271307402A12A7800E580307E01F4B1
:1003500030E502A12A885CA11253DACF207E034344
:10036000DA20307E0343DA10C271206102813253F9
:10037000DACF207E0343DA10307E0343DA20C2D87E
:10038000D27188578958C3E89555F8E99556F97B95
:10039000007E087A00C3E8948CE994005005755BF0
:1003A000008124882178A2E6A8216055C3E894C87A
:1003B000E994005008E4D2E4FB7A0A61FFC3E894B0
:1003C00068E994015008E4D2E3FB7A0F61FFC3E8C7
:1003D00094D0E994025008E4D2E2FB7A1E61FFC394
:1003E000E894A0E994055008E4D2E1FB7A3C61FF6F
:1003F000C3E89498E994085008E4D2E0FB7A787E48
:1004000000C3E89559FCE9955AFD30E70AECF4245D
:1004100001FCEDF43400FD755B00C3EC9AED9E50D9
:1004200003755B018859895A855755855856780256
:10043000A112C3E89527F8E99528F9307C0281F6E6
:10044000307B0281F6307A0281EF2075028155E916
:10045000FDE8FC8174E9C313F9E813F830790281EF
:10046000EFE9C313F9E813F830780281EFE9C31319
:0E047000FDE813FC20612CC3EC941CED9402FB
:10047E004002818BED701EC3EC94C850180529E51F
:10048E002970021529C3E529940A5002A12A755C28
:10049E0000D270A12AE529600215297400207F037D
:1004AE007896E624FAFEE43400FFC3EC9EFCED9F42
:1004BE00FD50067800790081F6C3EC94FFED9400B0
:1004CE00400678FF790081F6EC8572F0A4C5F0A2A3
:1004DE00F733F87900400302051278FF7900020520
:1004EE0012E9C313F9E813F8307C0EE9600278FFC5
:1004FE00C3E81338F8E43400F9C3E894FFE9940034
:10050E00400278FF885CD270206102A12A741FF429
:10051E00552F4BF52FC274EB7002D274752A4030F2
:10052E007403752A0A306102A13E20740353DAFE69
:10053E00207403752B20D0F0D0E0D0D0D2AD43E69E
:10054E001032790102056E790302056E790A0205F1
:10055E006E791E02056E796402056E79C802056E0B
:10056E007817E4D5E0FDD8FAD9F6227A147B780212
:10057E0005957A107B8C0205957A0D7BB402059554
:10058E007A0B7BC80205957902E4C282D5E0FDD2D2
:10059E0094D5E0FDC294D5E0FDD282D5E0FDE920F0
:1005AE00E002D28330E002D295E573D5E0FDE9207A
:1005BE00E002C28330E002C2957496D5E0FDD9C93F
:1005CE00EAF8D5E0FDD8FBDBBEC28222C37C007DFB
:1005DE000075F00005F0EA33FAEB33FB50F6EB133F
:1005EE00FBEA13FAC3E9FFE8FEE89AF8E99BF95033
:1005FE0004EFF9EEF8B3EC33FCED33FDD5F0DFED9F
:10060E00F9ECF822E889F08A20D2D4F8A9F07B0020
:10061E0030F70B7BFFF42401F8E9F43400F9E88598
:10062E0020F0A4ADF0F8E98520F0A4AFF0FEED2E99
:10063E00F974003FFA7C04C3EA13FAE913F9E813DC
:10064E00F8DCF48BF030F70AE8F42401F8E9F4341E
:10065E0000F9E889F0C2D4F8A9F0227882B6040332
:10066E00020708C3E55C9419401EE52D5406701868
:10067E00206E3678057994E7146007780A146002C4
:10068E007812C3E54198401F306E09856462756922
:10069E00FF756A01852224E4F544F545F546F547D4
:1006AE00F548C26E020708D26E7994E7147013E50E
:1006BE0023F43333F913F8E9540104F9E854FE0234
:1006CE0006FCE714147014E523F4333333F913F8EE
:1006DE00E9540304F9E854FC020704E523F4333328
:1006EE003333F913F8E954070404F9E854F8C394C2
:1006FE0040F8E99400F98844894522C3E54113F98D
:10070E00E54013F8C3E54498F8E54599F9500CC354
:10071E00E89480E994FF4016020740C3E8947FE90D
:10072E0094005003020740787F79000207407880DA
:10073E0079FF8849894A22E5492546F8E54A354731
:10074E00F9854A20E4300701F43548FA30E709C349
:10075E00EA94F0401502077EC3EA940F5003020795
:10076E007E78FF79FF7A0F02077E780079007AF0A3
:10077E00C3E5249561500AC374019524500B0207FA
:10078E009CE54A20E70E02079CE54A30E7068846BC
:10079E0089478A482278A5E6FAC3E54933F8E54A3F
:1007AE0033F9D112E930E70BC3E89480E994FF40A6
:1007BE0013E1D6C3E8947FE994005002E1D6787F26
:1007CE007900E1D6788079FFE820E715C3E5239814
:1007DE00F84009C3E8940140030207FD78010207BF
:1007EE00FDE8F424012523F840030207FD78FF8875
:1007FE004B2278A6E6FAA847A948120612E930E776
:10080E000CC3E89401E994FF4016020832C3E89441
:10081E00FFE99400500302083278FF790002083293
:10082E00780179FFE920E715C3E54B98F84009C335
:10083E00E8940140030208597801020859E8F424AB
:10084E0001254BF8400302085978FF88242278FFCF
:10085E00C26420693D206A12D264C3E541940A4005
:0F086E0009C3E52594405002C26479A1E76023D5
:10087D00E541601F74FF8541F0848539F0306A03CE
:10088D0075F005A4F8C5F0600278FFC3E8956450D3
:10089D0002A864886322C3E5409440E5419401E5D4
:1008AD006350031401B4046002F563227883E6F506
:1008BD0020120F3175E89012055075E890E5E8208B
:1008CD00ECFBA8BDA9BE120FD7756E55756F00C391
:1008DD00740013FD7455606613FC74552CFC740084
:1008ED003DFDECFAEDFBC3E89AE99B4014E56E245F
:1008FD0055F56EE56F3400F56FEA2CFAEB3DFB8094
:10090D00E5AE6EAF6FC3E56F13F9E56E13F8C3E98E
:10091D0013F9E813F87A03C3E913F9E813F8DAF7D2
:10092D00AA201A7009756E00756F0002094B1AEA3C
:10093D006008EE28FEEF39FFDAF88E6E8F6F2275A4
:10094D00E890227883E6FFE5E820ECF7A8BDA9BE84
:10095D000570C3E57094084052757000E9FA79A0EE
:10096D00E76044EA7007E571601B020986C3E895EC
:10097D00716010E5715006600C140209920460F963
:10098D00020992E571F571C3946D401B7561C0C389
:10099D0094044013756180C39404400B756140C38A
:1009AD009404400375610075BB0922EFC394016087
:1009BD001F7455601BC3E894FFE994035012C3E8FC
:1009CD00956EE9956F5009E561600C15610209E4BA
:1009DD00E561F460020561A861C3E524985002A8A1
:1009ED0024C3E89562400AA862E562F4600385625B
:1009FD006188258826E570B4070375BB1022743213
:100A0D0079A787F0A4C5F0A2F733F8C3E895614044
:100A1D0002A861882288248825882688642275404A
:100A2D00007541F022C2AF75C820A8CCA9CDAA3A55
:100A3D0030CF010A75C824D2AFAB3BAC3C883B89A3
:100A4D003CC3E89BF8E99C206908F9306702613ED8
:100A5D00419BAD3D8A3DF9EA9DFA600478FF79FF2F
:100A6D00AE3EAF3F8B3E8C3FA83BA93CC3E89EF802
:100A7D00E99FF9C3E54113FBE54013FAE82AF54078
:100A8D00E93BF54150067540FF7541FF41E5AA4030
:100A9D00AB41AC40AD417E047F02C3EB94044002F8
:100AAD001E1FC3EB940840021E1FC3ED13FDEC1374
:100ABD00FCDEF7C3EA9CFAEB9DFBEF6009C3E9137B
:100ACD00F9E813F8DFF7EA28FAEB39FB8A408B4196
:100ADD0050067BFF8B408B41C3EB94025002D267D3
:100AED003069047F0361107892E6FFC3E537948285
:100AFD0040110FC3E53794A040010FC3EF9406409A
:100B0D00027F057E02E541C4540FF9E541C454F05E
:100B1D00F8E540C4540F28F8C3E89EFAE99400FBA9
:100B2D004009C3EA9402EB940050047A02E4FB619D
:100B3D008AAA40AB41EBC4FEEAC4540F4EFCC3EA93
:100B4D009CFAEB9400FBC3E813C313F8EA28FAEB05
:100B5D003400FB8A408B41C3EB94024002C267789C
:100B6D0002EBC4FE7B00EAC4540F4EFAC3EA98FAB6
:100B7D004005C3940250027A027892E6FF3060027B
:100B8D00618A855192855293D26043E680C3E49A7F
:100B9D00F8E49BF93067028116E8FAE9FBD3E91313
:100BAD00FDE813FC88518952C3EF94036038EF20A0
:100BBD00E00DE82CF8E93DF9ECFAEDFB020BDFE86E
:100BCD0028F8E939F9C3E82402F8E93400F97AFE86
:100BDD007BFFC3EF9403400E8A538B54884D894E8F
:100BED008C4F8D50814A885389548A4D8B4E8C4F32
:100BFD008D503069127553F07554FF754FF0755067
:100C0D00FF7551F07552FF814AE8FAD3E813FC885D
:100C1D0051C3EF94036020EF20E007E82CF8ECFAC5
:100C2D008136E8282402F87AFEC3EF940340088A3F
:100C3D0053884D8C4F814A88538A4D8C4FE568C33C
:100C4D00335002646BF5683060028154753402D202
:100C5D006043E680E52D54066034A840A941C3E900
:0F0C6D0013F9E813F8C3E913F9E813F830690431
:100C7C00E92440F9C2AF53E67F759100C3E498F5BF
:100C8C0094E499F595759104D26043E680D2AF2235
:100C9C00D265754300752000306C03752040020C42
:100CAC00BBD265754300752040306C03752000780D
:100CBC00017901206720E52D54066002C265791484
:100CCC00E541C313700104F8C39414400278143046
:100CDC006904781B791B206010E543600C306903B4
:100CEC00D53404D26DA15E915C0543E59BF4544070
:100CFC00B52002A14830690908C3E8994001188160
:100D0C00E220650A08C3E899400281BB81E2C26512
:100D1C00C2AF53E67F7591003067127594007595DC
:100D2C00FE759104D26043E680D2AF81BBAE40AF7A
:100D3C0041C3E49EF594E49FF595A12DC3E533944E
:100D4C0001500281BB30650281BBD802A15C81E2FB
:100D5C00C26DC2AF53E67F7591008553948554954F
:100D6C00759104854D92854E93D26043E680D2AF47
:100D7C00E52D54066008206A020533020D9A306D89
:100D8C000D206C0A2065071581158102160F22783B
:100D9C00003064053065027801E53775F007A4F979
:100DAC00E5F028F5F0E9A2F013A2F113A2F213F585
:100DBC0037C394785003753778C3E53795384008B6
:100DCC00D266C283C294C295306002A1D4854F9280
:100DDC00855093D26043E68022207D16C2AF7542C7
:100DEC0002C282D280306202D295D2AF759F43028A
:100DFC000FD4C2AF754202C282D297306202D28344
:100E0C00D2AF759F43020FD4307243207D20C2AF06
:100E1C00754203900141757B04C295C29730620400
:100E2C00D294C132D282D2AF759F53020FD4C2AFCB
:100E3C00754203900141757B04C283C28030620409
:100E4C00D294C152D282D2AF759F33020FD4207D7F
:100E5C0017C2AF75420390011CC295306202D29446
:100E6C00D2AF759F53020FD4C2AF75420390011CD1
:100E7C00C283306202D294D2AF759F33020FD4205A
:100E8C007D16C2AF754204C280D297306202D294F2
:100E9C00D2AF759F33020FD4C2AF754204C297D242
:100EAC0080306202D294D2AF759F53020FD430724D
:100EBC0043207D20C2AF754205900130757B01C285
:100ECC0094C282306204D283C1D8D280D2AF759FD3
:100EDC0043020FD4C2AF754205900152757B80C29C
:100EEC0094C282306204D295C1F8D297D2AF759F6A
:100EFC0043020FD4207D17C2AF754205900112C278
:100F0C0094306202D283D2AF759F43020FD4C2AF2A
:100F1C00754205900126C2943062EBD295D2AF7522
:100F2C009F43020FD4207D16C2AF754206C297D2E2
:100F3C0082306202D283D2AF759F53020FD4C2AFFC
:100F4C00754206C280D282306202D295D2AF759FB2
:100F5C0033020FD4307243207D20C2AF7542019012
:100F6C000152757B80C283C280306204D295E17ECF
:100F7C00D297D2AF759F33020FD4C2AF7542019096
:100F8C000130757B01C295C297306204D283E19E19
:100F9C00D280D2AF759F53020FD4207D17C2AF758C
:100FAC004201900126C283306202D295D2AF759F66
:100FBC0033020FD4C2AF754201900112C295306258
:100FCC0002D283D2AF759F53C26622900110757BFB
:100FDC0000C283C294C295C280C282C297C26222EE
:100FEC00788076070876070876010876040876FF7D
:100FFC000876FF08760908760208760108760178EB
:10100C008C76010876000876B40876FF0876FF081F
:10101C0076FF0876030876FF0876010876FF0876D7
:10102C00250876D00876780876C80876040876FF06
:10103C0008760108760008767A08760A08760108A0
:10104C0076010876000876FF087600227887E6FF9E
:10105C00C272BF0302D2727888C27DE630E102D23E
:0F106C007DC27E7889E630E102D27EC3EF940226
:10107B006008758E01D27302108A758E00C27322BE
:10108B007880E6149000809378A5F67881E614902A
:10109B0000809378A6F67886E61490008D9378A757
:1010AB00F6789FE6F8700108C3E8941140027811B6
:1010BB00E82828F56B256B256B28F56C256B282804
:1010CB00F56D7886E6F539C39402500375390278CD
:1010DB009CE67538FFB402037538A0B4030375386A
:1010EB008278A3E61490009A93F566120FD722220A
:1010FB007896E6FA7897E6FB7888E6B40305C3EBB7
:10110B00940EFB307F047A007BFFC3EB9AFCC394F5
:10111B008250027C827572000572EC8572F0A4C35A
:10112B00E5F0947D40F222D27F11FB12055F7A002D
:10113B007B007C10120555E55C2AFA74003BFBDC46
:10114B00F37C04C3EB13FBEA13FADCF7FEC27F114B
:10115B00FB22E5EF20E6037520000520903FFFE51D
:10116B0020146006901DFF1460009304600375EF5C
:10117B001253D9BF7581C043FF8012055075EF0222
:10118B0043B203E5B3240220E70DF521E5E320E0AC
:10119B00068521B343E301120FD77580F275A40DB9
:1011AB0075F13F75D4DF75904F75A5B075F2F0757D
:1011BB00D50075A60175E241120FD7E4F8F6D8FDFC
:1011CB00756801120FEC12166678988673753001EC
:1011DB00C2AF12056912057912055F12058012055F
:1011EB005F12058712055F121789120569120569CF
:1011FB00120564C2AF78FA79FA308507D9FBD8F7B4
:10120B00021C001158118B11FA11FB78988673127E
:10121B000FD775881075890275C82475910475D818
:10122B004075A82275B80275E690759B80759D0078
:10123B0075D10E75BC5875BB0975BA1175E880125E
:10124B000550D2AF1208B975360053DACF207E03A2
:10125B0043DA20307E0343DA1043DA01C2D8C2717D
:10126B00120569D2617B037A0CE55B70077A0CDBA4
:10127B00030211FE12055F2070030211FEC270E51E
:10128B005CC3940240E1E52F541F855E5DF55EB5AE
:10129B005DD5DAD5C26153DACF207E0343DA203035
:1012AB007E0343DA10C2D8C27178A2E67008D274FA
:1012BB00E52F54E0F52FC2757529001205643074C3
:1012CB0009C3E529940A4002D275120555780230FC
:1012DB0074027800C3E55C9840F0C2AF1205791236
:1012EB000579120579D2AF120569754C00120555B7
:1012FB00788CE6C3940150030213CEE530C39401FE
:10130B0050030213CE207435C3E55C94FF500302E7
:10131B0013CEC2AF12058ED2AF120564C3E55C9437
:10132B000150EFC2AF12057912055A120579D2AFEF
:10133B00120564C3E55C94FF40E902180E7F05D2E9
:10134B007F11FB120564C2AFC27F11FBAE5CC3E51C
:10135B005C947FD2AF4076120550C2AF12058ED28D
:10136B00AFDFDC3132C3EE94057897F612056912C4
:10137B0016A81217917F0AD27F11FB120564C2AF18
:10138B00C27F11FBAE5CC3E55C947FD2AF50E6121B
:10139B000550C2AF12057912055A120579D2AFDF8B
:1013AB00D63132EE24037896F61205691216A8127E
:1013BB0017C012056411FBC3E55C94FF500261106A
:1013CB0002180EC3E55C954C4003855C4C1205641A
:1013DB0078017988E7B403027805C3E55C9840028D
:1013EB0041F8C2AF12058E12058E12058ED2AF12C6
:1013FB000569753000E4F531F5320531E531F470EE
:10140B003F0532789AE67819146012783214600D21
:10141B00787D14600878FA146003753200C3E532E6
:10142B0098401D120FD7120550153275310078995F
:10143B008673C2AF12058ED2AF789886731205648D
:10144B0012055AE52A700530740221FE78012074CA
:10145B00027806C3E55C9840A1120564E52A700387
:0F146B000211FEC2AF120FD7E4F522F523F524CC
:10147A00F525F526F567D2AF7885E6C333F565E439
:10148A00F544F545F546F547F548F570F52CF52D83
:10149A00F53775700875BB1012055012094CE5E84E
:1014AA0020ECFBA8BDA9BEE97001F88871120950A9
:1014BA0075700875BB101158C2AF7561FF120A0B1F
:1014CA00852261852262852263D2AF752201752445
:1014DA0001752501752601856069756A017888E6B6
:1014EA00B40307C27D307602D27DD268D2697533E1
:1014FA0000120F31120F60120A2B120A32120A2B33
:10150A00120A32120A2B120CAD120669120D9B1224
:10151A000DE5120A32120C9C306E0312070920677D
:10152A000312085C3067031208A3120D9B120E14F3
:10153A00120A32120CAD306E03120745120D9B12BD
:10154A000E8B120A32120C9C306E031207A3120D74
:10155A009B120EBA120A32120CAD306E0312080038
:10156A00120D9B120F31120A3212094C120C9C12E4
:10157A000D9B120F60120950120A3230692C8564D1
:10158A0061856462856069756A0179187A0CC3E5B8
:10159A0033994009C269D26A8A350215B4C3E55C37
:1015AA0094014003021510021617306A1D206C1AA6
:1015BA00E535147006C26AD26BA110F535C3E55C35
:1015CA0094014003021510021617753600C3E55F31
:1015DA0094014009856462856069756A0178FA79BF
:1015EA00A4E760027803C3E55F985021307404E5EC
:1015FA002A601A78F0306C058564617820C3E54169
:10160A00985002A1100536E55C6002C11A753600D1
:10161A00C2AF120FD77887E6FE760211587887EEA6
:10162A00F6E4F522F523F524F525F526F565752C5E
:10163A0000752D00D2AF120564120FD778A4E660A8
:10164A0006D283D294D295307406E52A700221FE1E
:10165A00788DE6C39401400241D58100901A0D7835
:10166A00201216EAE520B4A50CA31216EAE520B466
:10167A005A03021688120FEC1216A80216A7901A1D
:10168A000378807B0A1216EAA308DBF9901A0F780E
:10169A008C7B191216EAA308DBF9901A2822C2AF2A
:1016AA00121729121703901A00740E1216EFA37458
:1016BA00061216EFA374151216EF901A0378807BA0
:1016CA000A1216EEA308DBF9901A0F788C7B19120E
:1016DA0016EEA308DBF912173C12171A901A2822E1
:1016EA00E493F622E6438F01538FFD75EF0275B737
:1016FA00A575B7F1F0538FFE22438F02438F017510
:10170A00EF0275B7A575B7F1901A0DF0538FFC2249
:10171A00901A0D74A5D1EF901A0E745AD1EF227A4D
:10172A003079D07820901A40D1EAE520F709A3DA77
:10173A00F7227A3079D0901A40E7D1EF09A3DAF983
:10174A0022AB74A875BB01027980BB02027981BB06
:10175A0003027982BB04027994BB05027983BB0632
:10176A00027986BB07027992BB08027987BB090214
:10177A00799CBB0A027988BB0B027989E8F7227C3B
:10178A0005120569DCFB22C2AF1205791205801227
:10179A00058712058E12055A12057912058012055F
:1017AA008712058E12055A120579120580120587CD
:1017BA0012058ED2AF22C2AF12058E12058712050C
:1017CA008012057912055A12058E120587120580B4
:1017DA0012057912055A12058E1205871205801212
:1017EA000579D2AF22AE74AF75C2AF120579120570
:1017FA007912057912055ADEF212058E12055ADFA0
:10180A00F8D2AF221217911217891217897574012B
:10181A007575017576001217EF7C05AD5C120569C6
:10182A00C3ED955C70F5C3E55C9401400AC3E55CC1
:10183A0094FF403702185212174B1216A81217912A
:10184A00C2AF75EF12121789DCD10576C3E576941B
:10185A0003500280C11217890575E5741490009F20
:0E186A0093F808C3E57598500280A8121789FC
:101878001217890574C3E574940C50028094120FF2
:0C188800EC1216A8C2AF75EF12121789FF
:0319FD0002115D77
:101A00000E061507070104FFFF09020101A55A018F
:101A100000B4FFFFFF03FF01FF25D078C804FF01DA
:091A200000FF0A010100FF00FFB4
:101A400023416C69676E424C333558232020202097
:101A500023424C48454C4923463333302320202031
:101A60002020202020202020202020202020202076
:101C0000C2AFC2D353D9BF7581C043B20343FF8073
:101C1000752438752503B1C975EF0275E24043F1AB
:101C20002053A4DF75D4FFD2857DFA780379E67C52
:101C300010752200752300901DD67B0675249875BB
:101C400025013085028142208508D8FBD9F9DCF7CF
:101C500081B4308508D8FBD9F9DCF781B4B189E4C7
:101C600093A3C39A6004DDC381B4DBDBB17B600264
:101C7000812B7B08E493FAA3B15CDBF87A30B15C8A
:101C8000752200752300B17BEAFCEBFDC3ED94FEE9
:101C9000400EB17B8A278B28ED30E0048A828B834B
:101CA000B17B7AC270D8C3ED94FE601350CEBD00F4
:101CB00025EC60097520007521FF0200008100A855
:101CC00027A9280809D804D90281D3B17FEA89AAB3
:101CD000F281C50D81A0C3ED94035049EDA2E092BD
:101CE000007AC5C3E5829400E583941C50902000DF
:101CF00010438F02438F0175B7A575B7F1F030001F
:101D00001FA827A9280809438F01538FFDD804D99C
:101D100002A12089AAE275B7A575B7F1F0A3A10DBC
:101D2000538FFC817C7AC1BD030CE493A3FAB140CC
:101D3000DCF8B138817C817EAA22AB23B15CEBFA5E
:101D4000EA6222752608C3E52313F523E52213F57D
:101D50002250066323A0632201D526EAB1C9B1C986
:101D600075260AEAF4200102D285300102C285B14B
:101D7000C9C3134002C201D526EB22B17FEAFB2082
:101D80008502A17F308502A184752608AE24AF2587
:101D9000C3EF13FFEE13FEB1CDB1C9C3EA13308513
:101DA000024480FA30E703632201C3E52313F523DD
:101DB000E52213F52250066323A0632201D526D91C
:101DC000E52265236523F52222AE24AF250E0FDE22
:101DD000FEDFFCD20122424C48656C693437316326
:041DE000F3300601D5
:00000001FF
